:10000000E5C2FFC2FEC2FDC2FCC2FBC2FAC2F9C217
:10001000F8C269C3F6C2F5C2F4C2F3C2F2C2F1C2B9
:10002000F0C2EFC2EEC252474200000000000000E2
:1000300000000000000000000000000101000000BE
:1000400001000000010101000101010000010100A7
:100050000000010000000101010001010100000198
:100060000100000001000000010101000101010088
:100070000001010000000100000001010100010178
:1000800001000000524742207375627472616B7404
:10009000697600000000000000010001010101017B
:1000A0000101010100010101000101010001010143
:1000B0000101010101010001010100010101000133
:1000C0000101010101010101000101010001010122
:1000D0000001010101010101010100010101000113
:1000E00001005247422073657175656E7469656CD5
:1000F0006C00000000000001010000000100000091
:1001000001010100010101000001000000010100E6
:1001100000010101000101010000000000000101D7
:1001200001000101010000010100000001000001C7
:1001300001010001010100000001000000010100B7
:10014000524742207375627472616B7469762073D2
:1001500065712E0000010001010101010101010191
:100160000001010100010100010101010101010182
:100170000100010101000101010101010101010171
:100180000101000101010001010101010101010161
:1001900000010100010101000101010101005247BC
:1001A000422065696E7A2E2073636877656C6C6592
:1001B0006E6400000100000000000000000001006B
:1001C000000001000000010000000000000000002D
:1001D000010000000100000001000000000000001C
:1001E000000001000000010000000100000000000C
:1001F00000000000010000000100000100000100FB
:1002000001000100010001000100010001000200E5
:1002100002000200020002000200020002000200CE
:1002200002000200020003000300030003000300B9
:1002300003000300040004000400040004000400A0
:100240000500050005000500050006000600060083
:100250000600070007000700080008000800090062
:1002600009000A000A000A000B000B000C000C0039
:100270000D000D000E000F000F0010001100110006
:1002800012001300140015001600170018001900C2
:100290001A001B001C001D001F002000210023006D
:1002A00024002600280029002B002D002F003100FB
:1002B0003400360038003B003D004000430046005B
:1002C00049004C004F00530057005B005F00630083
:1002D00067006C00700075007B00800086008C0059
:1002E000920098009F00A600AD00B500BD00C500BB
:1002F000CE00D700E100EB00F50000010B01170173
:10030000240130013E014C015B016A017A018B013D
:100310009C01AF01C201D601EA01000217022E02C0
:10032000470261027C029802B502D402F40216036D
:1003300039035D038303AB03D50300042D045D047F
:100340008E04C204F80430056B05A805E8052B06E9
:100350007106BA0606075607A90700085B08B90820
:100360001C098309EF09600AD50A500BD10B560C02
:10037000E20C740D0D0EAC0E520F0010B51073117F
:1003800038120713DF13C014AB15A116A117AD184F
:10039000C419E91A1A1C581DA51E00206B21E5225C
:1003A00071240E26BD278029562B412D422F5A310C
:1003B0008933D1353338B03A493D0040D542CB4539
:1003C000E2481C4C7A4FFF52AC56825A845EB362AC
:1003D0001267A26B66706075927A0080AA85958B11
:1003E000C3913798F59EFEA558AD04B508BD66C506
:1003F00024CE44D7CCE0C0EA25F5FFFF44757263F4
:10040000686C6175667A6569742033206D696E0069
:10041000007544757263686C6175667A65697420ED
:1004200032206D696E00004E44757263686C6175B0
:10043000667A6569742039302073656B003B4475BA
:100440007263686C6175667A6569742036302073F2
:10045000656B002744757263686C6175667A6569BF
:10046000742034302073656B001A44757263686CB5
:100470006175667A6569742033302073656B00148A
:1004800044757263686C6175667A65697420323090
:100490002073656B000D44757263686C6175667AD4
:1004A0006569742031352073656B000A4475726389
:1004B000686C6175667A6569742031302073656B8C
:1004C000000744757263686C6175667A65697420AB
:1004D000342073656B000003526F7400000000004D
:1004E00000000000000000000000000000FF00000D
:1004F000FFFFFF477275656E0000000000000000FE
:10050000000000000000000000FF00FFFFFF426C41
:100510006175000000000000000000000000000005
:100520000000000000FFFFFFFF57656973730000C4
:100530000000000000000000000000000000FFFFBD
:10054000FFFFFFFF47656C62000000000000000035
:10055000000000000000000000FFFF00FFFFFF564A
:10056000696F6C65747400000000000000000000FA
:1005700000000000FF00FFFFFFFF416D6265720099
:10058000000000000000000000000000000000FF6C
:10059000FFDFFFFFFF547565726B69730000000099
:1005A0000000000000000000000000FFFFFFFFFF50
:1005B0004F72616E676500000000000000000000DF
:1005C0000000000000FFC000FFFFFF0011241FBE5D
:1005D000CFE5D4E0DEBFCDBF11E0A0E6B0E0E8EFAC
:1005E000FAE102C005900D92AA39B107D9F712E0DD
:1005F000AAE9B1E001C01D92A631B107E1F702D02E
:1006000079CAFECCFF920F931F938CE050D18FD10B
:1006100063D27CD2789417D410E000E0FF24FA94DF
:1006200001C000E080917000833049F0843161F0B6
:10063000823091F4112309F452C011500FC01530CB
:1006400009F44FC01F5F0AC0002319F400D101E074
:1006500005C0F9D300E002C08F3F11F0F0927000A6
:100660000130F9F61230D1F0133028F4112351F093
:100670001130C1F60DC01430E9F01430A8F0153077
:1006800089F627C0E4D08BE991E066E270E017C0FC
:10069000DED08BE991E064E870E011C0D8D08BE93E
:1006A00091E062EE70E00BC0D2D08BE991E060E4A3
:1006B00071E005C0CCD08BE991E06EE971E04EE5C8
:1006C00050E0CCD98BE991E0DAD08BE991E0B7D258
:1006D000A9CFBDD080E690E0D2D06ED2A3CF15E0F6
:1006E000BDCF10E0BBCF1F920F920FB60F92112417
:1006F0002F933F934F935F936F937F938F939F932A
:10070000AF93BF93EF93FF9380919A018F5F8732EE
:10071000A8F063B3617080E025D163B3627081E0BB
:1007200021D166B3617082E01DD166B3627083E04F
:1007300019D166B3647084E015D180E080939A018A
:10074000FF91EF91BF91AF919F918F917F916F91A9
:100750005F914F913F912F910F900FBE0F901F907F
:100760001895662311F0909A01C0909891988B9AF1
:100770008C9A8D9A8E9A969895989498939887FDCE
:10078000969A86FD959A85FD949A84FD939A929AFD
:1007900000C09298969895989498939883FD969A0D
:1007A00082FD959A81FD949A80FD939A929A00C059
:1007B0009298939A949A959A969A0895882311F00C
:1007C000909A01C09098919A8B988C988D988E9859
:1007D000929A00C0839B02C080E101C080E08499AE
:1007E00080628599806486998068929800C0929A08
:1007F00000C083998160849982608599846086991C
:1008000088609298089580E0D9DF87FDFCCF85E06D
:100810008A95F1F780E0D2DF08951F93182FF3DF58
:10082000812F60E09EDF1F9108951F93182FEBDF4B
:10083000812F61E096DF1F910895662311F480589F
:1008400001C08054EADF0895DEDF90E0089581E082
:10085000E4DF089582E0E1DF08951F93182FD3DFCE
:100860001A3041F4803410F080E001C080E48058F8
:10087000D4DF03C0812F61E074DF1F910895CF930F
:10088000DF93EC0101C0E9DF89918823E1F7DF9173
:10089000CF910895CF93DF93EC0101C0DEDFFE011D
:1008A000219684918823D1F7DF91CF9108950F93FA
:1008B0001F93082F889A899A8A9A8B9A8C9A8D9A74
:1008C0008E9A88E592E028EC30E0F9013197F1F753
:1008D0000197D9F7949A929A00C09298929A00C080
:1008E00092989498969A929A00C092989698929A12
:1008F00000C0929810EA812F8A95F1F788E08DDF89
:100900001A95F1F7A4DF80EA9FE00197F1F786E0FE
:1009100084DF802F82DF1F910F9108951F9310E0D5
:1009200080E29BDF1F5F1431D9F71F910895A098D3
:10093000A89AA198A99AB898C09AB998C19ABA9851
:10094000C29A92E09093FB019093FE0110920102F3
:100950001092040281E08093070293BF89B78160FF
:1009600089BF0895582F83E0589FF0011124E75064
:10097000FE4F318190E0662309F491E0918342813A
:100980002081832F8095892341F0413019F0952FE4
:1009900020E01DC09FEF20E020C0892F832321F09D
:1009A0002E3F58F42F5F09C09095932331F04130CA
:1009B00069F42F3FD1F0952F03C0413039F49FEFF8
:1009C000203559F4952F905F2FEF07C09FEF4230ED
:1009D00021F42C3311F4952F2DE2809170008F3F7C
:1009E00011F490937000208308959FEFF6CF2FE0CD
:1009F000AB9897FDAB9AAC9AAB98AC98880F991FBF
:100A00002150B1F7AB9897FDAB9AAD9AAC9AAB98E1
:100A1000AD98AC9808952FE0AB9897FDAB9AAC9A3F
:100A2000AB98AC98880F991F21502130A9F7AB984B
:100A300097FDAB9AAD9AAC9AAB98AC9896FDAB9AF1
:100A4000AC9AAB98AD98AC980895A0E0B0E0EAE21B
:100A5000F5E023C86C01E62E7FE0F72E80E090E001
:100A6000C6DFFA948BE0F816C9F78601F801838592
:100A7000EE2051F4882319F480E090E00DC0D82FC7
:100A8000C0E0CE01019708C0E82FF0E0EE0FFF1F95
:100A9000E450FE4F85919491AADFFA9401501040E2
:100AA000FF2021F7F6018081EE2049F4882319F414
:100AB00080E090E00CC0982F80E0019708C0E82FFC
:100AC000F0E0EE0FFF1FE450FE4F85919491A3DFFD
:100AD000CDB7DEB7E8E0FDC7AB98AC98AD98A39A68
:100AE000A49AA59ABB9A85B5896185BD88E083BD26
:100AF0000895FA01861749F09081681718F4892F34
:100B0000815002C0892F8F5F808308951092080260
:100B10001092090208956095681710F080E008951A
:100B2000861B0895ABE1B0E0E7E9F5E0B8C7BC018A
:100B30008E010F5F1F4FC8014BE150E08FD780E05F
:100B400061E07BDEEBDE80E061E077DEC80197DE0E
:100B50000E89598D5095E02EE51AB88D4B8D409534
:100B6000FB2EF41AAF893A8D30951A2F131BEAE049
:100B7000F2E020E0822F63E07AD7992321F4501726
:100B800060F48E2D0DC0913021F44B1730F48F2D71
:100B900007C0923031F43A1710F080E001C0812F85
:100BA00080832F5F31962C3029F78AE092E061E054
:100BB0004CDF6B96E6E08FC7FF920F931F938091F7
:100BC00009022BE1829FC001112488529B4FAADFAA
:100BD0001BE188E0F82E0FEF8091700085303CF427
:100BE00082304CF5882331F0813001F50CC084311E
:100BF000E9F421C080910902882319F4F0920902D6
:100C00000CC0815008C080910902883019F41092FC
:100C1000090203C08F5F8093090280910902819FBE
:100C2000C001112488529B4F7DDF02C08F3FA1F28B
:100C300000937000D1CF1F910F91FF900895A9E10B
:100C4000B0E0E4E2F6E01FC72C016091080286E103
:100C5000689FB001112464507C4F8E010F5F1F4FBD
:100C6000C80146E150E0FAD680E061E0E6DD56DEFC
:100C700080E061E0E2DDC80102DE4F8A652CAAE077
:100C8000B2E0F2018589882311F08FEF01C080E086
:100C90008D93369682E0A631B807A1F77724D2016A
:100CA000A35ABF4FB98FA88F01C0772422243324C1
:100CB000872C9924E5E1F0E08E0E9F1E840C951C94
:100CC00080917000853044F482300CF0B9C08823E4
:100CD00031F08130C1F515C08431A9F5B1C08091E2
:100CE0000802882321F4F9E0F093080203C0815040
:100CF000809308026091080286E1689FB001112488
:100D000010C080910802893019F41092080203C0C3
:100D10008F5F809308026091080296E1699FB0019D
:100D2000112464507C4FCE01019646E150E096D6E6
:100D300080E061E082DDF2DD80E061E07EDDCE0119
:100D400001969DDD02C08F3F19F0AFEFA0937000B8
:100D5000EAE0F2E0A4018F89962D9C01B901B4E08C
:100D6000B71528F0DA012C9111969C9109C0B5E0D5
:100D70007B1679F4DB015A962C915A9755969C91E3
:100D8000291739F08081921710F4815001C08F5FCC
:100D900080836A5F7F4F31964A5F5F4FB2E0E631F2
:100DA000FB07E9F6CF010C97E88DF98D60814DDEE8
:100DB0006E8970E080E090E0E7D35B016C0120E099
:100DC00030E04AEF54E419D27B018C0120E030E09E
:100DD00040E85FE35DD388231CF461E070E01FC04E
:100DE000C801B70120E03FEF4FE757E4FBD21816E8
:100DF0009CF4C601B50120E030E040E251E4FDD1B1
:100E000038D006C088EC90E00197F1F7615070404F
:100E100061157105B9F706C0C801B7012AD0CB0129
:100E20000197F1F70894211C311CFFEF2F163104B4
:100E300009F046CF739486E0781609F037CF35CFA6
:100E40006996E2E13CC603DD81E790E018DD80E0D1
:100E500061E0F3DC86E890E012DDEAE0F2E0119276
:100E600082E0E631F807D9F7CF010C9760E0EDDDBD
:100E70000895EF92FF920F931F937B018C0120E066
:100E800030E040E05FE4D9D288237CF0C801B701AC
:100E900020E030E040E05FE45ED125D39B01AC016F
:100EA000205030404040504805C0C801B7011BD316
:100EB0009B01AC01B901CA011F910F91FF90EF9006
:100EC0000895A0E0B0E0E6E6F7E0DDC5DC012B0127
:100ED000FA019C91923008F439C1EB01888182308B
:100EE00008F433C1943069F4843009F02FC11196AD
:100EF0009C9111978981981709F428C1A2E9B0E063
:100F000025C1843009F421C18230A9F4923009F05E
:100F10001DC19A01AD0188E0EA010990AE01E90125
:100F200009929E018150C1F7E201898111969C913D
:100F30008923818308C1923009F407C112962D904C
:100F40003C901397EB018A819B811496AD90BD90E4
:100F5000CD90DC901797EC80FD800E811F81910170
:100F6000281B390BB90137FF04C066277727621B9E
:100F7000730B603271050CF061C0121613066CF52C
:100F800037014801062E04C096948794779467949D
:100F90000A94D2F721E030E040E050E004C0220F94
:100FA000331F441F551F6A95D2F7215030404040EF
:100FB00050402E213F214023512321153105410569
:100FC000510521F021E030E040E050E079018A0154
:100FD000E628F728082919293CC0232BD1F1260E31
:100FE000371E35014601062E04C0969487947794E7
:100FF00067940A94D2F721E030E040E050E004C06A
:10100000220F331F441F551F6A95D2F721503040DD
:10101000404050402A213B214C215D2121153105C2
:101020004105510521F021E030E040E050E0590158
:101030006A01A628B728C828D9280BC082159305AD
:101040002CF01C01AA24BB24650103C0EE24FF245C
:10105000870111969C91D20111968C91981709F4F1
:1010600045C0992339F0A80197012A193B094C0979
:101070005D0906C0A60195012E193F09400B510BD1
:1010800057FD08C011823382228224833583468330
:1010900057831DC081E0818333822282882799276C
:1010A000DC01821B930BA40BB50B84839583A68371
:1010B000B7830DC0220F331F441F551F2483358370
:1010C000468357838281938101979383828324810E
:1010D000358146815781DA01C9010197A109B1091A
:1010E0008F5F9F4FAF4FBF4328F30BC09183338275
:1010F0002282EA0CFB1C0C1D1D1DE482F582068376
:10110000178383E08083248135814681578157FF8F
:101110001AC0C901AA2797FDA095BA2F81709070B7
:10112000A070B0705695479537952795822B932BD5
:10113000A42BB52B84839583A683B7838281938167
:10114000019693838283DF0101C0D201CD01CDB727
:10115000DEB7E2E1B4C4A0E2B0E0E0EBF8E09FC4A7
:1011600069837A838B839C832D833E834F83588747
:10117000E9E0EE2EF12CEC0EFD1ECE010196B7013A
:101180009CD38E010F5E1F4FCE010596B80195D3FB
:101190008A8991E089278A8BC701B801AE01475E31
:1011A0005F4F8FDEB5D2A096E6E095C4A0E2B0E036
:1011B000EBEDF8E074C469837A838B839C832D8381
:1011C0003E834F835887F9E0EF2EF12CEC0EFD1E85
:1011D000CE010196B70171D38E010F5E1F4FCE0174
:1011E0000596B8016AD3C701B801AE01475E5F4FEB
:1011F00068DE8ED2A096E6E06EC4A0E2B0E0E2E047
:10120000F9E041C469837A838B839C832D833E8379
:101210004F835887CE010196BE01675F7F4F4DD344
:10122000CE010596BE016F5E7F4F47D39985923000
:1012300088F089898230C8F0943019F4823051F4F2
:1012400004C0843029F4923081F482E990E0C6C071
:10125000923049F420E09A858A89981321E02A8700
:10126000CE010996BBC0823049F420E09A858A8974
:10127000981321E02A8BCE014196B0C02D843E8484
:101280004F8458886D887E888F88988CEE24FF2440
:101290008701AA24BB24650140E050E060E070E0D3
:1012A000E0E0F0E0C10181709070892BE9F0E60C7C
:1012B000F71C081D191D9A01AB012A0D3B1D4C1D81
:1012C0005D1D80E090E0A0E0B0E0E614F7040805C2
:1012D000190520F481E090E0A0E0B0E0BA01A90196
:1012E000480F591F6A1F7B1FAA0CBB1CCC1CDD1C9E
:1012F00097FE08C081E090E0A0E0B0E0A82AB92AFB
:10130000CA2ADB2A3196E032F10549F0660C771CD7
:10131000881C991C5694479437942794C3CFFA8518
:10132000EA892B893C898B859C85280F391F2E5F84
:101330003F4F17C0CA0181709070892B61F01695DC
:101340000795F794E79480E090E0A0E0B0E8E82A01
:10135000F92A0A2B1B2B76956795579547952F5F92
:101360003F4F77FDE7CF0CC0440F551F661F771F17
:1013700017FD4160EE0CFF1C001F111F2150304073
:10138000403090E0590790E0690790E4790760F3F6
:101390002B8F3C8FDB01CA018F779070A070B070EB
:1013A00080349105A105B10561F447FD0AC0E1143F
:1013B000F1040105110529F0405C5F4F6F4F7F4F2D
:1013C00040781A8EFE1711F081E08A8F4D8F5E8F64
:1013D0006F8F78A383E0898FCE01499699D1A0962B
:1013E000E2E16DC3A8E1B0E0E7EFF9E058C369833B
:1013F0007A838B839C832D833E834F83588789E038
:10140000E82EF12CEC0EFD1ECE010196B70155D24F
:101410008E010F5E1F4FCE010596B8014ED2898511
:10142000823038F08989823020F0C701B801BDD2FE
:1014300001C08FEF6896E6E04EC3A8E1B0E0E2E2BB
:10144000FAE02DC369837A838B839C832D833E834B
:101450004F83588789E0E82EF12CEC0EFD1ECE015B
:101460000196B7012AD28E010F5E1F4FCE0105965D
:10147000B80123D28985823038F08989823020F002
:10148000C701B80192D201C08FEF6896E6E023C38E
:10149000A8E1B0E0EDE4FAE002C369837A838B83CC
:1014A0009C832D833E834F83588789E0E82EF12C5F
:1014B000EC0EFD1ECE010196B701FFD18E010F5E2D
:1014C0001F4FCE010596B801F8D18985823038F0DA
:1014D0008989823020F0C701B80167D201C081E05C
:1014E0006896E6E0F8C2ACE0B0E0E8E7FAE0DBC21C
:1014F00069837A838B839C83CE010196BE016B5FE7
:101500007F4FDBD18D81823061F1823050F18430A8
:1015100021F48E81882351F12EC02F81388537FD2B
:1015200020C06E812F3131051CF06623F9F023C0F5
:101530008EE190E0821B930B29853A854B855C8573
:1015400004C056954795379527958A95D2F7662317
:10155000B1F050954095309521953F4F4F4F5F4FDB
:101560000EC020E030E040E050E009C02FEF3FEF38
:101570004FEF5FE704C020E030E040E050E8B90101
:10158000CA012C96E2E0ABC2A8E0B0E0E9ECFAE0D8
:1015900082C27B018C01611571058105910519F4E9
:1015A00082E089835FC083E089838EE1C82ED12CDD
:1015B000DC82CB82ED82FE820F831887C801B701DF
:1015C00058D0FC013197F7FF3BC0222733272E1B51
:1015D0003F0B57016801022E04C0D694C794B794FC
:1015E000A7940A94D2F740E050E060E070E081E018
:1015F00090E0A0E0B0E004C0880F991FAA1FBB1FB5
:101600002A95D2F70197A109B1098E219F21A02324
:10161000B1230097A105B10521F041E050E060E061
:1016200070E04A295B296C297D294D835E836F8395
:1016300078878EE190E08E1B9F0B9C838B8312C07A
:10164000309781F00E2E04C0EE0CFF1C001F111FFE
:101650000A94D2F7ED82FE820F831887CE1ADF0A32
:10166000DC82CB821A82CE01019652D02896EAE023
:101670002EC2EF92FF920F931F937B018C0180E0AB
:10168000E81680E0F80681E0080780E0180788F493
:101690008FEFE816F1040105110531F028F088E01C
:1016A00090E0A0E0B0E017C080E090E0A0E0B0E003
:1016B00012C080E0E81680E0F80680E0080781E0CC
:1016C000180728F088E190E0A0E0B0E004C080E1D5
:1016D00090E0A0E0B0E020E230E040E050E0281BE5
:1016E000390B4A0B5B0B04C016950795F794E794EA
:1016F0008A95D2F7F701E656FF4F8081281B310902
:1017000041095109C9011F910F91FF90EF90089570
:10171000DF92EF92FF920F931F93FC01E480F5801C
:1017200006811781D1808081823048F480E090E08A
:10173000A0E1B0E0E82AF92A0A2B1B2BA5C08430CF
:1017400009F49FC0823021F4EE24FF24870105C0F4
:10175000E114F1040105110519F4E0E0F0E096C090
:10176000628173819FEF623879070CF05BC022E8D9
:101770003FEF261B370B2A3131052CF020E030E0FB
:1017800040E050E02AC0B801A701022E04C07695BF
:101790006795579547950A94D2F781E090E0A0E0CD
:1017A000B0E004C0880F991FAA1FBB1F2A95D2F76B
:1017B0000197A109B1098E219F21A023B123009790
:1017C000A105B10521F081E090E0A0E0B0E09A0130
:1017D000AB01282B392B4A2B5B2BDA01C9018F7700
:1017E0009070A070B07080349105A105B10539F4F6
:1017F00027FF09C0205C3F4F4F4F5F4F04C0215C63
:101800003F4F4F4F5F4FE0E0F0E02030A0E03A075D
:10181000A0E04A07A0E45A0710F0E1E0F0E0790107
:101820008A0127C06038710564F5FB01E158FF4F5C
:10183000D801C7018F779070A070B0708034910587
:10184000A105B10539F4E7FE0DC080E490E0A0E009
:10185000B0E004C08FE390E0A0E0B0E0E80EF91E35
:101860000A1F1B1F17FF05C016950795F794E794ED
:10187000319687E016950795F794E7948A95D1F706
:1018800005C0EE24FF248701EFEFF0E06E2F67958F
:1018900066276795902F9F77D794DD24D7948E2F56
:1018A0008695492F462B582F5D29B701CA011F91F4
:1018B0000F91FF90EF90DF900895FC01DB014081D4
:1018C00051812281622F6F7770E0221F2227221F11
:1018D0009381892F880F822B282F30E0991F992719
:1018E000991F11969C93119721153105A9F5411562
:1018F00051056105710511F482E037C082E89FEF60
:1019000013969C938E9312979A01AB0167E0220F76
:10191000331F441F551F6A95D1F783E08C930DC088
:10192000220F331F441F551F12968D919C911397C0
:10193000019713969C938E931297203080E038077E
:1019400080E0480780E4580758F314962D933D93A0
:101950004D935C93179708952F3F310579F4411506
:1019600051056105710519F484E08C93089564FFB5
:1019700003C081E08C9312C01C9210C02F573040DE
:1019800013963C932E93129783E08C9387E0440F39
:10199000551F661F771F8A95D1F7706414964D9373
:1019A0005D936D937C93179708951F93DC01FB0162
:1019B0009C91923008F447C08081823008F443C083
:1019C000943051F411961C91843099F58181682FDF
:1019D00070E0611B71093FC0843021F0923031F416
:1019E0008230B9F18181882389F12DC011961C9133
:1019F00011978230F1F081811817D9F412962D9148
:101A00003C911397828193818217930794F0281752
:101A10003907BCF014968D919D910D90BC91A02D2D
:101A20002481358146815781281739074A075B078A
:101A300018F4112341F00AC082179307A407B507D1
:101A400040F4112319F061E070E005C06FEF7FEF03
:101A500002C060E070E0CB011F910895FB01DC0142
:101A600002C005900D9241505040D8F70895991B3F
:101A700079E004C0991F961708F0961B881F7A9585
:101A8000C9F7809508952F923F924F925F926F927F
:101A90007F928F929F92AF92BF92CF92DF92EF92FE
:101AA000FF920F931F93CF93DF93CDB7DEB7CA1B7F
:101AB000DB0B0FB6F894DEBF0FBECDBF09942A88AA
:101AC000398848885F846E847D848C849B84AA8452
:101AD000B984C884DF80EE80FD800C811B81AA81DF
:101AE000B981CE0FD11D0FB6F894DEBF0FBECDBFAA
:081AF000ED010895F894FFCF09
:101AF8006B6F6E7374616E74652046617262650007
:101B0800FF4F4E2F4F46462064727565636B656EB6
:101B180020667565720045696E736368616C7465EB
:101B28006E00000000000000000000010202030334
:101B38000303040404040404040405050505050559
:101B48000505050505050505050506060606060637
:101B5800060606060606060606060606060606061D
:101B68000606060606060606060607070707070707
:101B780007070707070707070707070707070707ED
:101B880007070707070707070707070707070707DD
:101B980007070707070707070707070707070707CD
:101BA80007070707070707070707080808080808B7
:101BB800080808080808080808080808080808089D
:101BC800080808080808080808080808080808088D
:101BD800080808080808080808080808080808087D
:101BE800080808080808080808080808080808086D
:101BF800080808080808080808080808080808085D
:101C0800080808080808080808080808080808084C
:101C1800080808080808080808080808080808083C
:0A1C28000808080808080808080862
:00000001FF
